S00B0000737476684F484A68E6
S113000009C008C007C063C15BC104C003C06AC0A3
S113001001C000C0F8940FED0DBF002701BB09E437
S113002008BB07BB00E808B90CE009B900E205BF4A
S1130030EE27DD2755246624FF240DE5E02ED9BFE5
S1130040C09A08E90AB9C69B05C001E15D9BFECFD1
S11300500CB9C69878948895FECF0FEFDBBD0ABD26
S1130060C098002408E408BF09BF0BEC0EBDE9CF1B
S113007078948895F894FF20D9F7DBBD2ABCC09802
S113008008E408BF09BF0BEC0EBDDBCF789488955C
S1130090F894FF20D9F7DBBDDABDE0E6CE2FC09897
S11300A000E408BF09BFCDCF552466247894889511
S11300B0F894FF20D9F70FEF0BBD0ABD08E008BF85
S11300C009BF09E00EBD7894C398BBCF7894889596
S11300D0F894FF20D9F702E00EBDF0948F2CE0E6EF
S11300E0CE2FAFCFF7FE24C0579887FE78940CB17B
S11300F0FBB1F4FD58C0F3FD56C0F894F9B7FD13F5
S113010008C007D0F894F8E0F8BFF9BF86991895AD
S1130110F3C07894FC2FFE1BFA95F7FDF458FD13F9
S113012001C041C0FE110EC0F3E1FCB9C69A0AC079
S11301300CB1FBB1F871B9F5E03670F4FD1201C0F1
S113014030C0FA94FF270193FCED08E9F8940AB94A
S1130150EF131895E0E6189572FC16C070FC23C0E6
S11301600D1305C07394CE131895002721C071FC9C
S11301700BC00154C0F00031B0F4043028F4D02F87
S1130180DD0FDD0F0D2BDD27CE13C4CFFEB5F770C9
S113019009F6F0E8FFBDFBE0FEBDFF27FBBD0ABC8E
S11301A0B9CF093028F0F89400270CB955246624F7
S11301B0C39A9924DD27D9BFD3BFDFBDDEBDDDBD22
S11301C0DCBDFFEDFDBFF02FF063FCB9EE27083076
S11301D0E8F5043068F4023020F4FF2400FF2FCF48
S11301E03CCFF3E0FF2E00FF43CFF39477244ECFB0
S11301F0F2E0FF2E063018F5C09A00FF67CF56CF05
S113020036FC0FC024B445B4C39A09E40EBD189556
S1130210351848F2E32DE295EF7029F23394632CFC
S11302203BC034B405B532180409069537940695D5
S11302303794662079F4552059F7532C2DC000FFCC
S113024033CF02E0702E0024FF2425CFF4E0FF2EEC
S11302507F2E1CCFE0EF3A94351880F0F0E1762C35
S113026022247A94872CF69549F0720C77943714EB
S1130270C0F3EF0F7394272C782CF5CF992011F449
S11302809E2E0AC0E2959E225D9BFECF9CB89924C7
S113029008940908190838F0EE27C39809E00EBD40
S11302A01895E0E4ECB9C39A9924FF24EFEDEDBF6F
S11302B0EE27DD27D9BFDFBDDEBDDDBDDCBDBFCE92
S11302C00FB507FD4CC00EB5087F0EBD18953EB4A2
S11302D033FC2DC087FC10C0C39AD0E43D263EBC3D
S11302E0DD278A9422F090FEC3989694189508947A
S11302F00D0A1D0AB0F21895CE1302C0D9BF189585
S11303009990CC3D09F4C0E6DC2FDE1BDA95D7FDCD
S1130310D458DD3528F0C69B03C0D1E1DCB9C698BA
S1130320C398D2E4DEBDD8E08D2EDD27189537FEC4
S113033067CFDDBDDCBD0BEC0EBD04B5002059F06C
S1130340F02F01E4FF2339F00395F01520F0039515
S1130350F11508F003955D9BFECF0CB9189506FFC7
S11303601AC000E80FBD72FC0CC071FC11C0DE2F76
S1130370E42DE695E6950081ED2FDD27DBBD0ABD72
S11303801895D2E07D26DE2FE42D4294EC70F1CF57
S1130390DBBD4ABC189506E0701206C000EC0FBD28
S11303A0DE2FE42DE370E7CFCE1305C0002772FEE5
S11303B070FCFECE88CF00EC0FBD4990042D71FC7B
S11303C006C00370DE2FE02F0081ED2FDD27DBBD9B
S11303D00ABDCC3D09F4C0E6FC2FFE1BFA95F7FDDF
S11303E0F458FD3528F0C69B189501E10CB9C69860
S10503F018955A
S9030000FC
